S01300005344495F4D61696E4170702E737265632C
S11300000C942D010C9453010C9453010C94530142
S11300100C9453010C9453010C9453010C9453010C
S11300200C9453010C9453010C9453010C945301FC
S11300300C9453010C94D0090C9453010C94530167
S11300400C9453010C9453010C9453010C945301DC
S11300500C9453010C9453010C9453010C945301CC
S11300600C9453010C9435120C9483120C94530188
S11300700C9453010C9453010C9453010C945301AC
S11300800C9453010C9453010C9453010C9453019C
S11300900C9453010C9453010C9453010C9453018C
S11300A00C9453010C9453010C9453010C9453017C
S11300B00C9453010C9453010C94030A0C945301B3
S11300C00C9453010C9453010C9453010C9453015C
S11300D00C9453010C9453010C9453010C9453014C
S11300E00C9453010C9453010C9453010C9453013C
S11300F00C9453010C9453010C9453010C9453012C
S11301000C9453010C9453010C9453010C9453011B
S11301100C9453010C9453010C9453010C9453010B
S11301200C9453010C9453010C9453010C945301FB
S11301300C9453010C9453010C9453010C945301EB
S11301400C9453010C9453010C9453010C945301DB
S11301500C9453010C9453010C9453010C945301CB
S11301600C9453010C9453010C9453010C945301BB
S11301700C9453010C9453010C9453010C945301AB
S11301800C9453010C9453010C9453010C9453019B
S11301900C9453010C9453010C9453010C9453018B
S11301A00C9453010C9453010C9453010C9453017B
S11301B00C9453010C9453010C9453010C9453016B
S11301C00C9453010C9453010C9453010C9453015B
S11301D00C9453010C9453010C9453010C9453014B
S11301E00C9453010C9453010C9453010C9453013B
S11301F00C9453010C94A70F0C947410380B3B0B04
S11302003E0B410B440B470B4A0B0C943E0B0C94D6
S1130210A8020C942F030C94470B0C9446040C94E2
S113022097050C94BE010C94B4010C943B0B0C94F4
S1130230410B0C94C4010C94380B0C944A0B0C9491
S1130240440B0C9412040C94BC010C943B030C94CA
S1130250C1020C9418030C94BA0111241FBECFEFF1
S1130260CDBFDFE3DEBF00E00CBF18BE19BE1ABE6F
S11302701BBE10E2A0E0B0E2ECE8F7E200E00BBF46
S113028002C007900D92A63BB107D9F71BBE23E22B
S1130290A6EBB0E201C01D92A034B207E1F70E94C0
S11302A055010C94C4130C94000087E08093A200C1
S11302B07894EAE2F3E210821182128213821482A9
S11302C081E085830E94C4120E94271380E090E09D
S11302D00895E0E0F6E081E0858382E0858384E0B0
S11302E0858380E1858380E2858380E4858380E85B
S11302F08583089581E080930606089584E08093C1
S113030006060895E0E0F6E084E0858380E18583D5
S113031080E2858380E4858380E88583089580E195
S113032080930606089580E180930506089580E28F
S113033080930606089580E280930506089580E47C
S113034080930606089580E8809306060895009732
S113035021F482E0809306060895883E934019F4C0
S113036082E08093050608958091CC21815080938A
S1130370CC21089580E0089580E008956CED71E249
S113038080E00E94A71108951092CC211092D821E8
S11303901092D921EEECF1E281EA808380E281833C
S11303A0128213821482158282E090E086839783FE
S11303B010861186ECEDF1E280E092ECA1E0B0E071
S11303C080839183A283B3831482158288E0868319
S11303D0BF0180E00E94A71180E00E94931188234E
S11303E029F09091CC219F5F9093CC210895FF92A6
S11303F00F931F93CF93DF931F92CDB7DEB78091F6
S1130400B92081119EC00E94650D882351F000918E
S1130410BA201091BB200E94720D0817190759F4D5
S113042090C00091BA201091BB200E946D0D081756
S1130430190709F486C08FB78983F894198100914C
S1130440BC20E02FF0E0EE0FFF1FE354FF4D80814E
S11304509181892B09F58091B6209091B72001965E
S11304608093B6209093B7200E94650D811107C038
S11304708091B6209091B7208436910558F00E945F
S1130480650D882349F08091B6209091B720803281
S1130490934010F41FBF55C01092B6201092B7209D
S11304A08091B820811106C081E0011180E0809321
S11304B0BC2004C081E0011180E0082F81E080931A
S11304C0B9201FBF10E0F801EE0FFF1FE354FF4DEA
S11304D0FF24F394808191818034910509F4F12CF7
S11304E0FF2091F00E94650D882339F00E94720D5F
S11304F08093BA209093BB200BC00E946D0D809313
S1130500BA209093BB2004C01092BA201092BB2052
S1130510F801EE0FFF1FE354FF4D20813181A80144
S11305200024569547950794569547950794542F5C
S1130530402D4E535F4D08EA12E06F2D81E80E9472
S1130540570E0F90DF91CF911F910F91FF90089557
S1130550811116C02091BC2081E090E0222311F08B
S113056080E090E0880F991FFC01E354FF4D108256
S113057011821092B8201092B92080E00E94F701F5
S1130580089580E00E94F70108950F931F938091CE
S1130590DA2181111FC02091D8213091D921809175
S11305A0D6219091D72128173907A1F0862F2091C1
S11305B0D8213091D9212093D6213093D72108E135
S11305C013E02AE030E04EEC51E260E00E94570E66
S11305D08093DA211F910F910895CF93DF931F9297
S11305E0CDB7DEB78FB78983F8942981662359F094
S11305F08091D8219091D921482B592B4093D8210F
S11306005093D9210CC08091D8219091D921409543
S11306105095482359234093D8215093D9212FBF73
S113062062E880E00E94C5020F90DF91CF910895A7
S11306301092DA218091D8219091D92183788093E6
S1130640D8219093D921EEECF1E2808591858378CD
S113065080879187642F80E00E94C502089580916D
S1130660CB2181508093CB218091CB210E949A1180
S11306701092CA210895809130238823CCF4807687
S11306808032F1F5809131238132E1F58091362376
S1130690909137230797C1F5E0E3F3E28CED91E203
S11306A08087918787E090E08287938781E008952F
S11306B08076803259F580913123803219F082326C
S11306C0B9F026C08091362390913723079711F50E
S11306D0E0E3F3E28EEB91E0848795878CED91E281
S11306E08087918787E090E08287938781E00895EF
S11306F060913223617080E00E949F1181E008952F
S113070080E0089580E0089580E0089580E00895F1
S113071080E0089580E0089540E150E061E080E0E9
S11307200E94ED02089540E450E061E080E00E9400
S1130730ED020895CF93DF931F92CDB7DEB78FB745
S11307408983F89449812091432130914421E09197
S11307504521F0E0EE0FFF1FEA5BFE4D80819181A1
S11307604FBF821B930B0F90DF91CF9108950E948E
S11307709A0321E0892B09F420E0822F08950F9336
S11307801F93CF93DF931F92CDB7DEB78FB78983C3
S1130790F89499812091452180914221811110C0C2
S11307A06091432170914421022F10E0F801EE0F73
S11307B0FF1FEA5BFE4D408151816417750718F4F1
S11307C09FBF80E029C0109243211092442181E010
S11307D0211180E08093452181E0809342219FBFD5
S11307E080E00E94B703882319F080E00E942D1254
S11307F0A801002456954795079456954795079464
S1130800542F402D465B5E4D06E414E020E430E0B6
S113081061E082E00E94570E0F90DF91CF911F910B
S11308200F9108951092CB211092B9201092B82004
S11308301092BC20EDEBF0E210821182128213823E
S11308401092BA201092BB2080E00E94F70110920F
S1130850422110924521E6E4F1E2108211821282D3
S11308601382109243211092442180E00E94BF031E
S1130870882359F09091CB219F5F9093CB21909145
S1130880CB21913011F49093CA2108950F931F93B3
S113089081112AC080914521E1E08111E0E0842F9B
S11308A061157105A9F4F0E00024F695E795079425
S11308B0F695E7950794FE2FE02DAF01465B5E4D5C
S11308C006E414E020E430E061E00E94570E0CC01E
S11308D0F0E0EE0FFF1FEA5BFE4D60837183109220
S11308E0422180E00E94BF031F910F91089580E090
S11308F00E94B7030895EF92FF921F93CF93DF9363
S11309001F92CDB7DEB711E08091E221893009F062
S113091010E040E050E08FB78983F894A9812091DA
S11309204321309144218091452190E0FC01EE0F58
S1130930FF1FEA5BFE4D60817181AFBF2617370749
S113094030F08091CA218111E6CF90E022C0FC01F1
S11309500024F695E7950794F695E7950794FE2FFE
S1130960E02DE20FF31FE65BFE4D80817A01E82A59
S11309702F5F3F4F209343213093442180E00E9416
S1130980BF03112321F05E2D442710E0C4CF8E2D28
S11309909F2D0F90DF91CF911F91FF90EF900895BD
S11309A080E00E947B040895CF93DF931F92CDB71C
S11309B0DEB78FB78983F89499818091BC20E82FA2
S11309C0F0E0EE0FFF1FE354FF4D2081318120340E
S11309D0310589F44091B92041110DC04091B820EE
S11309E0411109C021E02093B820811120E0209317
S11309F0BC2020E030E09FBF80E490E0821B930B9A
S1130A000F90DF91CF9108950E94D40421E0892BA7
S1130A1009F420E0822F089580E00E9404050895DF
S1130A20FF920F931F93CF93DF931F92CDB7DEB73F
S1130A30F62E172F01E08091E221893009F000E0C1
S1130A4080E00E940405811107C08091CA218111B0
S1130A50F7CF80E090E02DC08FB78983F894298187
S1130A60E091BC20F0E0DF01AA0FBB1FA354BF4DEF
S1130A708D919C911197AC014F5F5F4F4D935C93A7
S1130A800024F695E7950794F695E7950794FE2FCD
S1130A90E02D8E0F9F1FFC01EE53FF4DF0822FBF00
S1130AA0002329F0F12E110F110B00E0C9CF81E0D2
S1130AB090E00F90DF91CF911F910F91FF900895D7
S1130AC0BC0180E00E9410050895E091E821F091B6
S1130AD0E9210190F081E02D228133812E0F3F1F07
S1130AE0FC014081E40FF11DE217F307B8F48181A2
S1130AF08430B9F0861309C005C081818430A1F027
S1130B00861303C08E2F9F2F08958081E80FF11D57
S1130B10E217F30790F380E090E0089580E090E01E
S1130B20089580E090E0089580E090E00895809139
S1130B3032238F770E94670D08959091EA219923BB
S1130B4081F1E091E821F091E9210190F081E02D1B
S1130B509481891740F5E093E621F093E7212281FF
S1130B6033812E0F3F1FE217F307F8F4918194307D
S1130B7061F49281981309C09381961306C0E0939F
S1130B80E621F093E72181E008959081E90FF11DBA
S1130B90E217F30758F3E093E621F093E72180E0AE
S1130BA0089580E0089580E0089580E00895EF922C
S1130BB0FF921F93CF93DF93C82F60E00E949D059F
S1130BC0182F882391F1A091E821B091E921EC2F0D
S1130BD0F0E0EE0FFF1F12968D919C911397E80F92
S1130BE0F91FE080F180D7011696ED91FC911797DB
S1130BF01995682F8C2F0E949D05182F8823A9F022
S1130C00C091E621D091E72165E0CE010E946505FF
S1130C10EC01892B21F08A810E946C0FF5CFD7015A
S1130C201296ED91FC9113971995812FDF91CF9135
S1130C301F91FF90EF9008951F93CF93DF93182F88
S1130C400E949D05882349F1C091E621D091E721B6
S1130C5065E0CE010E946505EC01892B49F04C81C9
S1130C605D816B818A810E947C0D8111F1CF15C059
S1130C70A091E821B091E921E12FF0E0EE0FFF1FF0
S1130C8012968D919C911397E80FF91F0190F081B2
S1130C90E02D0190F081E02D1995DF91CF911F9106
S1130CA00895CF938091EA218823C9F0E091E82147
S1130CB0F091E9210190F081E02D8481882379F07D
S1130CC0C0E08C2F0E94D705CF5FE091E821F0911E
S1130CD0E9210190F081E02D8481C81790F31092EE
S1130CE0EA2181E090E08093EE219093EF21CF916F
S1130CF00895CF938091EA21882349F1A091E821B6
S1130D00B091E921ED91FC91119784818823F9F048
S1130D10C0E0EC2FF0E0EE0FFF1F12968D919C9136
S1130D201397E80FF91F0190F081E02D0084F185FD
S1130D30E02D309709F01995CF5FA091E821B0918B
S1130D40E921ED91FC9111978481C81710F3CF919B
S1130D5008950F931F93CF93DF93E0E3F3E212869A
S1130D6013861486158616861786808188230CF0D0
S1130D7070C220913623309137232115310509F0B3
S1130D806DC263C28F7109F0AAC09091312396306D
S1130D9081F0983009F498C09111A1C02230310536
S1130DA009F0D9C162E070E08EEE91E20E94750D07
S1130DB05AC28091322390913323292F3327223032
S1130DC03105B1F024F42130310541F0BBC12330A9
S1130DD03105F1F12F30310561F1B4C18091142056
S1130DE090911520DC016C9170E00E94750D5DC03E
S1130DF0E0911420F09115202189821708F0ABC1ED
S1130E009927880F991F880F991FE0911620F09158
S1130E101720E80FF91F80819181FC0162817381A1
S1130E200E94750DE0913823F091392382E081838B
S1130E303CC08091182090911920009709F48BC12F
S1130E40DC0112966D917C9113970E94750D2DC053
S1130E5099278130910579F038F0029709F07BC128
S1130E6088E990E22FE00AC064E070E082EB90E24F
S1130E700E94750D1AC088EA90E229E0382FAAE78B
S1130E80B0E2E82FF92F819190E08D939D938E2FFE
S1130E90831B8217C0F3622F660F6E5F6093782006
S1130EA070E088E790E20E94750DE0E3F3E286814A
S1130EB09781228533858217930708F0D4C18093E4
S1130EC03A2390933B23CFC12130310509F043C12C
S1130ED061E070E08AEE91E20E94750DC4C1813038
S1130EE0F1F5909131239A30D1F52130310509F093
S1130EF032C18091EA21882309F42DC1C0913423A1
S1130F00D09135230091E8211091E921D801ED9188
S1130F10FC918481C81708F01EC160E08C2F0E94E8
S1130F209D05882309F417C1CE019927880F991FBD
S1130F30D8011296ED91FC911397E80FF91F0190D7
S1130F40F081E02D86819781FC0119958093EC2135
S1130F5061E070E08CEE91E20E94750D84C18230F4
S1130F6009F0F9C0809131238111EEC0223031059E
S1130F7009F0F1C0809134230E94040E90E0809324
S1130F80E4219093E52162E070E084EE91E20E9416
S1130F90750D69C18F7109F086C09091312393302A
S1130FA009F4D4C018F49130A1F07DC0953019F043
S1130FB0993039F178C08091362390913723892B69
S1130FC009F0C9C087E995E080933C2390933D23C1
S1130FD04AC18091362390913723892B09F0BBC0F5
S1130FE08091322390913323019709F0B4C080910A
S1130FF0EE219091EF218D7F8093EE219093EF214C
S113100032C18091362390913723892B09F0A3C0F4
S11310100E946A0D882309F49EC0209132233091E6
S113102033233327E0911420F0911520818990E037
S11310308217930708F48FC00E94510680913223CF
S1131040909133238093EA21882309F40CC19927D2
S11310508150904C880F991F880F991FE09116209A
S1131060F0911720E80FF91FE093E821F093E921AC
S11310700190F081E02D8481882309F4F4C0C0E05C
S113108060E08C2F0E941C06882309F464C0CF5FA3
S1131090E091E821F091E9210190F081E02D848133
S11310A0C81770F3E0C08130F1F4909131239B3084
S11310B0D1F48091362390913723892B09F04BC0CA
S11310C08091EA21882309F446C0E0E3F3E2C48175
S11310D0D2818C2F0E94D7058823E9F16D2F8C2FA4
S11310E00E941C0636C08230B1F5809131238130D4
S11310F019F0833091F02CC08091362390913723DE
S1131100892B49F58091322390913323892B19F54A
S1131110809134230E941F0E1CC08091362390912D
S11311203723892BC1F48091322390913323892B67
S113113091F4C0E3D3E28C810E94220F8C810E943F
S1131140890F07C080E005C080E003C080E001C0D3
S113115080E0811189C0809130238F71813081F5C5
S11311608091EA21882361F1009134231091352381
S1131170C091E821D091E921E881F981848108179F
S1131180F8F460E0802F0E949D058823C9F0F801DF
S1131190FF27CF01880F991FEA81FB81E80FF91F10
S11311A0C081D181EE81FF811995682F802F0E9423
S11311B09D05882329F0EC81FD811995811154C086
S11311C0809130238F71823009F041C08091EA21EF
S11311D08823B9F1A091E821B091E921ED91FC9126
S11311E011978481882379F1C0E0EC2FF0E0EE0FB1
S11311F0FF1F12968D919C911397E80FF91F0081A0
S11312001181D8011696ED91FC9117971995682FC5
S11312108C2F0E949D05882339F1D8011496ED91F5
S1131220FC911597199581111FC0CF5FA091E821FA
S1131230B091E921ED91FC9111979481C917A8F21D
S113124013C080E011C080E00FC080E00DC080E0DA
S11312500BC0982F907609F07ECF9CCE982F907675
S113126009F079CF8FCD81E0DF91CF911F910F915C
S11312700895CF93DF93E091F021F091F1218481DF
S113128083FF08C08860848383E0838386EF809330
S1131290FA2183C0982F947131F083E083838FEF18
S11312A08093FA217AC086FF43C0C0EFD1E2AA81BD
S11312B0BB818C819D8114962D913C911597821749
S11312C093076CF49C012F5F3F4F2093F4213093DC
S11312D0F521A80FB91F11968C9187835EC0809168
S11312E0F6219091F72118962D913C911997821728
S11312F09307C8F42091F821222321F0868181608C
S113130086834BC016962D913C911797AC014F5F85
S11313105F4F4093F6215093F721D901A80FB91FCD
S11313208C9187833AC083E083831092FA2135C07D
S1131330882384F5A0EFB1E21296CD91DC91139746
S113134016968D919C911797288539858217930756
S1131350D8F46E817F819C012F5F3F4F2093F6214B
S11313603093F7214781DB01A80FB91F4C9388857F
S113137099852817390718F482E083830EC087E023
S113138083831092FA2109C083E0838389EF8093D9
S1131390FA2103C08BEF8093FA21DF91CF91089556
S11313A01F920F920FB60F92112408B60F9218BE17
S11313B009B60F9219BE0BB60F921BBE2F933F9323
S11313C04F935F936F937F938F939F93AF93BF9349
S11313D0EF93FF930E943909FF91EF91BF91AF9171
S11313E09F918F917F916F915F914F913F912F9139
S11313F00F900BBE0F9009BE0F9008BE0F900FBE4A
S11314000F901F9018951F920F920FB60F921124F0
S113141008B60F9218BE09B60F9219BE0BB60F92FA
S11314201BBE2F933F934F935F936F937F938F9341
S11314309F93AF93BF93EF93FF930E943909FF915A
S1131440EF91BF91AF919F918F917F916F915F9138
S11314504F913F912F910F900BBE0F9009BE0F90AB
S113146008BE0F900FBE0F901F901895CF93DF9377
S11314701F921F92CDB7DEB7811126C09091282309
S11314809923F9F090912B23911101C0FFCF9FB7BD
S11314909A83F8942A81EAE2F3E29181915091834C
S11314A02FBF0FC090912B239F3F09F4FFCF9FB70D
S11314B09983F8942981EAE2F3E291819F5F918311
S11314C02FBF8093282305C090912823992351F39B
S11314D0F8CF0F900F90DF91CF9108950F93E8EC20
S11314E0F4E080818F7D808380818F7D8083ECEF29
S11314F0F2E202E005931092FE221092FF2200E233
S1131500069300E40693E4EFF2E200E2069300E4BB
S11315100693E0E3F3E21486158616861786128690
S113152013861092E4220F9108950F9385E080931F
S1131530E422EDEFF2E204E00593E5EFF2E204E0E9
S113154005930F9108950F9383E08093E422109202
S1131550FE221092FF22ECEFF2E202E006930F91DA
S11315600895E0913C23F0913D23309709F01995BB
S113157008950F93CF93DF938091E422833029F46D
S11315800E94B10A0E946E0A5EC08091E02290918E
S1131590E122C0913A23D0913B23C81BD90B71F5AA
S11315A02091E2223091E322820F931F8093E22262
S11315B09093E322209136233091372382179307A7
S11315C021F08091FB21882341F084E08093E42280
S11315D0E4EFF2E202E0069336C0E0913E23F0919C
S11315E03F23309799F01995882381F01092E022D7
S11315F01092E122C0913A23D0913B23C034D1050B
S113160028F01092FB21C0E4D0E003C081E0809375
S1131610FB21E8EEF2E2C68BD78B8091E022909119
S1131620E1222091382330913923280F391F208F4C
S1131630318FC80FD91FC093E022D093E122ECEF81
S1131640F2E202E00693DF91CF910F910895FC013D
S11316508181E82FE7708E2F90E0FC013197E7300D
S1131660F105D8F48827E250FF4F8F4F0C94B21342
S113167080E190E0089580E290E0089580E490E0B5
S1131680089580E890E0089580E091E0089580E076
S113169092E008958FEF93E0089588E090E0089534
S11316A0282F2F7030E0220F331F082E000C990BC7
S11316B08827990F881F9927820F931F02979C01EF
S11316C0220F331F220F331F220F331F820F931F4A
S11316D084589D4D08950F93CF938091CC0480FF3F
S11316E068C081E08093CC04E4EFF2E200E8069362
S11316F0ECEFF2E200E806938093CA04E4EFF2E22E
S113170000E106938091E422882339F083508230EB
S113171010F40E94B10A0E946E0A8091F622909100
S1131720F722089709F047C088E0E0EAF2E2A0E374
S1131730B3E201900D928A95E1F7E8ECF4E0808140
S1131740806280838081806280830E94A906C82F82
S1131750811104C00E94950AC1E02EC080913023FB
S1131760882374F41092E2221092E3221092E02271
S11317701092E12282E08093E4220E94B90A1CC004
S11317808091362390913723892B19F40E94A30A60
S113179013C01092E2221092E3221092E0221092DF
S11317A0E12281E08093E422E4EFF2E202E0069396
S11317B003C0C0E001C0C1E08C2FCF910F91089508
S11317C08F929F92AF92BF92DF92EF92FF920F930C
S11317D01F93CF93DF93D82E0E94500B8C01BD2C06
S11317E0BB1CBB24BB1CCD2DCF70D0E0CC0FDD1FA8
S11317F0CB0DD11DCE01880F991F880F991F880F1B
S1131800991F9C012C503D4D7901C9010E94270B61
S11318104C01BB2009F47BC0FE01EE0FFF1FEE0F4D
S1131820FF1FEE0FFF1FE851FD4D22893389D801B8
S113183015968D919C911697820F931F15968D93F3
S11318409C93169713962D913C91149782179307A6
S113185009F447C0281B390B2115B4E03B0740F0BD
S11318602FEF33E0C901B4010E947C13281B390B0C
S1131870F801808181FF0AC0C901B4010E947C1370
S113188041E0892B09F040E0842F01C080E0D801B9
S11318909C9180FB91F99C93FE01EE0FFF1FEE0FCC
S11318A0FF1FEE0FFF1FE851FD4D128A138A268792
S11318B0378711962D913C91129715968D919C9195
S11318C01697820F931FCC0FDD1FCC0FDD1FCC0F9B
S11318D0DD1FC850DD4D88839983F70102E006932C
S11318E0E8C0D8018C9181FFD1C08D7F8C93CC0F3F
S11318F0DD1FCC0FDD1FCC0FDD1FC851DD4D1A8A53
S11319001B8A1E861F86F70102E00693D2C0FE01E1
S1131910EE0FFF1FEE0FFF1FEE0FFF1FE851FD4DEF
S1131920A684B784D8018C9182FF1BC01196ED91D7
S1131930FC91129715962D913C91169713968D91C3
S11319409C911497B4010E947C13B0E4DB9EB00117
S1131950112464547E4DAC01CF01820F931F0E9469
S1131960BB13F801258136812A0D3B1D258336835F
S1131970838194818217930768F485839683CC0FBF
S1131980DD1FCC0FDD1FCC0FDD1FC851DD4D8A8953
S11319909B897CC0FE01EE0FFF1FEE0FFF1FEE0FB1
S11319A0FF1FE851FD4D428953894A155B0509F033
S11319B06DC02817390709F469C0AC01421B530BE9
S11319C09A01211554E0350758F02FEF33E0C9018F
S11319D0B4010E947C13D901A81BB90BCD0108C026
S11319E0C901B4010E947C13F901E81BF90BCF0172
S11319F0FE01EE0FFF1FEE0FFF1FEE0FFF1FE8515A
S1131A00FD4D168617868815990500F5D8018C9129
S1131A1084608C93B0E4DB9EC001112484549E4DF9
S1131A20FE01EE0FFF1FEE0FFF1FEE0FFF1FE8502A
S1131A30FD4D80839183CC0FDD1FCC0FDD1FCC0FB8
S1131A40DD1FC851DD4D8A8A9B8A1CC0F801418183
S1131A50528125813681240F351FFE01EE0FFF1FB1
S1131A60EE0FFF1FEE0FFF1FE850FD4D2083318363
S1131A70CC0FDD1FCC0FDD1FCC0FDD1FC851DD4D9A
S1131A808A8B9B8BF70102E0069313C0D8018C91DB
S1131A9080FF0FC08E7F8C931796ED91FC91189761
S1131AA0309739F015966D917C9116974D2D80E005
S1131AB01995DF91CF911F910F91FF90EF90DF90D7
S1131AC0BF90AF909F908F90089580E00895809389
S1131AD0C30408958091C3040895809124239091B0
S1131AE02523089580E090E00895E0E3F3E2808701
S1131AF09187628773870895282F2F7030E0220F13
S1131B00331F082E000C990B8827990F881F9927DB
S1131B10820F931FFC01EE0FFF1FEE0FFF1FEE0F4E
S1131B20FF1FE851FD4D2585207C09F069C06370D5
S1131B30613011F018F404C020EC03C020E801C0A7
S1131B4020E440385105E9F050F440325105A9F041
S1131B5040345105A1F040315105D9F40CC0411570
S1131B6032E0530791F04F3F33E0530781F04115C2
S1131B70514079F408C041E00DC042E00BC043E09D
S1131B8009C044E007C045E005C046E003C047E0A3
S1131B9001C040E0FC01EE0FFF1FEE0FFF1FEE0F30
S1131BA0FF1FE851FD4D158636E03487242B258729
S1131BB0FC01EE0FFF1FEE0FFF1FEE0FFF1FE8519A
S1131BC0FD4D2585207C203C69F4FC01EE0FFF1FB0
S1131BD0EE0FFF1FEE0FFF1FE851FD4D2585277007
S1131BE0273081F0880F991F880F991F880F991F3C
S1131BF0FC01E851FD4D85858062858781E008956B
S1131C0080E0089581E00895E82FEF70F0E0EE0F92
S1131C10FF1F082E000C990B8827990F881F9927FE
S1131C20E80FF91FEE0FFF1FEE0FFF1FEE0FFF1F50
S1131C30E851FD4D858582FB882780F908950F932F
S1131C40282F2F7030E0A901440F551F282F082E8C
S1131C50000C330B2227330F221F3327240F351F89
S1131C60A901440F551F440F551F440F551FFA0176
S1131C70EC50FD4D01E00693FA01E851FD4D9585C8
S1131C8092FF12C0FA01E851FD4D95859B7F95871F
S1131C900E94500BFC01808180FF06C08E7F8083F0
S1131CA00780F085E02D199581E00F9108955F92EA
S1131CB06F927F928F929F92AF92BF92CF92DF9258
S1131CC0EF92FF920F931F93CF93DF931F92CDB7A1
S1131CD0DEB7782E662E4A0159010E94500B6C0122
S1131CE0572C551C5524551C872D8F70E82EF12C2C
S1131CF0EE0CFF1CE50CF11CF701EE0FFF1FEE0FBD
S1131D00FF1FEE0FFF1FE851FD4D8585807C09F410
S1131D1084C0F701EE0FFF1FEE0FFF1FEE0FFF1F32
S1131D20E851FD4D8585807C803C61F0F701EE0F24
S1131D30FF1FEE0FFF1FEE0FFF1FE851FD4D8585BE
S1131D4082FD6DC08FB78983F8948981F6019081F3
S1131D5090FF03C08FBF512C63C0F6019081916046
S1131D6090838FBF81829282A382B482158216826D
S1131D7007831087611006C091E0A114B10419F023
S1131D8090E001C091E0F601808190FB81F98B7FA6
S1131D908083552061F0F701EE0FFF1FEE0FFF1F48
S1131DA0EE0FFF1FE851FD4D128A138A30C0F70170
S1131DB0EE0FFF1FEE0FFF1FEE0FFF1FE851FD4D4B
S1131DC08585807C803CB1F4C701880F991F880FFA
S1131DD0991F880F991F8C509D4D0E94270BBC01A1
S1131DE0C5010E947C13892B29F0F60180818E7F26
S1131DF0808316C0F701EE0FFF1FEE0FFF1FEE0FDB
S1131E00FF1FE851FD4D16861786128A138A872D07
S1131E100E94E00B5524539403C0512C01C0512C53
S1131E20852D0F90DF91CF911F910F91FF90EF902F
S1131E30DF90CF90BF90AF909F908F907F906F90E6
S1131E405F900895FF920F931F93CF93DF93182F02
S1131E50F82EFF1CFF24FF1CC82FCF70D0E0CC0F3E
S1131E60DD1FCF0DD11D0E94500BDC01FE01EE0FD2
S1131E70FF1FEE0FFF1FEE0FFF1FEC50FD4D02E0A2
S1131E8005938C9180FF22C08E7F8C931796ED91E1
S1131E90FC9118973097D1F0FF2059F0CC0FDD1F3B
S1131EA0CC0FDD1FCC0FDD1FC851DD4D6A897B8946
S1131EB00AC0CC0FDD1FCC0FDD1FCC0FDD1FC851B6
S1131EC0DD4D6E857F85412F81E01995DF91CF919E
S1131ED01F910F91FF900895CF93C82F0E94220F56
S1131EE0EC2FEF70F0E0EE0FFF1F8C2FCC0F990B4F
S1131EF08827990F881F9927E80FF91FEE0FFF1FF6
S1131F00EE0FFF1FEE0FFF1FE851FD4D1586CF9119
S1131F100895E82FEF70F0E0EE0FFF1F282F082E32
S1131F20000C330B2227330F221F3327E20FF31F3A
S1131F30EE0FFF1FEE0FFF1FEE0FFF1FE851FD4DC9
S1131F409585946095870E94220F81E008951F92E1
S1131F500F920FB60F92112408B60F9218BE09B64D
S1131F600F9219BE0BB60F921BBE0F932F933F9384
S1131F704F935F936F937F938F939F93AF93BF938D
S1131F80EF93FF938091CB04882344F480E88093FB
S1131F90CA040E9479060E948A118EC08091CB04E3
S1131FA082FF22C084E08093CA048091FC2286FFD1
S1131FB083C08091CC0481FD7FC00E946B0B811192
S1131FC07BC08091E422813019F40E94A30A74C07A
S1131FD0843009F071C0EDEFF2E204E00593E5EF1F
S1131FE0F2E204E0059368C08091CB0481FF5FC0F6
S1131FF082E08093CA048091F42286FF5DC08091C0
S1132000CC0481FD59C00E946B0B811155C0809195
S1132010E422823041F484E08093E422E4EFF2E2AB
S113202002E0069349C0833009F046C0EDEFF2E2C6
S113203004E00593E5EFF2E204E005933DC080E19E
S11320408093CA0481E00E94220F81E80E94220F3B
S11320500E9451061092C304E8EEF2E2158696E05F
S1132060948783E48587158A948B858B80EA92E232
S1132070808B918B0E946E0A1FC08091CB0486FFD7
S113208009C080E48093CA0480E00E94360A0E945A
S1132090841112C08091CB0485FF0EC080E280932E
S11320A0CA0481E00E94360A0E94871105C080910B
S11320B0CB0484FFE2CFC3CFFF91EF91BF91AF91E7
S11320C09F918F917F916F915F914F913F912F914C
S11320D00F910F900BBE0F9009BE0F9008BE0F908A
S11320E00FBE0F901F9018951F920F920FB60F926C
S11320F0112408B60F9218BE09B60F9219BE0AB67B
S11321000F921ABE0BB60F921BBE0F931F932F9301
S11321103F934F935F936F937F938F939F93AF936B
S1132120BF93CF93DF93EF93FF938091CC0481FD12
S113213004C00E946B0B8111CAC082E08093CC045E
S11321408091C5048195880FE4EFF2E2E81BF10960
S113215020813181245F3242369527953695279523
S113216036952795822F869520FD02C090E001C008
S113217090E8890FE82FEF70F0E0EE0FFF1F282F93
S1132180082E000C330B2227330F221F3327E20FB4
S1132190F31FDF01AA0FBB1FAA0FBB1FAA0FBB1F90
S11321A0A851BD4D1C969C9195FF91C0EE0FFF1F49
S11321B0EE0FFF1FEE0FFF1FEC50FD4D00E20693E4
S11321C081117EC08091E422843029F40E94B10AF6
S11321D00E946E0A7CC00091F6221091F722809131
S11321E03A2390913B23C091E022D091E1229E01B9
S11321F0200F311F8217930718F48C010C1B1D0B41
S11322008091382390913923A80160EA72E28C0FFF
S11322109D1F0E94BB13C00FD11FC093E022D09317
S1132220E1220034110569F48091E2229091E322C5
S11322308C0F9D1F209136233091372382179307EB
S113224090F0E0E3F3E2C287D3870684F785E02DBC
S1132250309731F01995811103C00E94950A37C057
S11322600E94A30A34C080913A2390913B23C8175B
S1132270D90709F5E0913E23F0913F23309719F4F3
S11322800E94950A24C01995811103C00E94950AE1
S11322901EC02091E2223091E3228091E0229091AD
S11322A0E122820F931F8093E2229093E322109203
S11322B0E0221092E122E4EFF2E202E0069307C08A
S11322C0803819F40E94B90A02C00E94E00BFF9101
S11322D0EF91DF91CF91BF91AF919F918F917F91BA
S11322E06F915F914F913F912F911F910F910F909B
S11322F00BBE0F900ABE0F9009BE0F9008BE0F9040
S11323000FBE0F901F9018950E94690108950E94B6
S11323107A01089580912923882321F00E946D0D6C
S11323200E94A701089591E0909329230E9413121B
S113233081E00895109229230E94241208956623AF
S113234019F00E947E0108950E9482010895FF926F
S11323500F931F93CF93DF938B01FB018481823012
S113236021F46894FF24F3F801C0F12CF80185816D
S1132370813031F0823039F4FF2DF062FF2E03C03A
S11323808F2D8063F82EF8018681863049F018F489
S11323908530A9F00DC0873039F0893069F008C064
S11323A0FF2DF160FF2E0BC08F2D8260F82E07C029
S11323B0EF2DE360FE2E03C0FF2DF760FF2E60E1DA
S11323C083E00E94D412C0EAD8E0FD82F801808143
S11323D09181A281B381880F991FAA1FBB1F880F07
S11323E0991FAA1FBB1F9C01AD01220F331F441F5D
S11323F0551F60E079E08DE390E00E949013DA01CC
S1132400C9010196A11DB11DB695A795979587950C
S11324109C01215031092E833F83DF91CF911F917D
S11324200F91FF90089560E183E00E94D412E0E4EC
S1132430F6E088E0818384E08283E0EAF8E08CE1DE
S1132440848380E38383089560E183E00E94EA1239
S1132450E0EAF8E01382148208958091A3088823A7
S113246019F083E38093A30808951F920F920FB687
S11324700F92112408B60F9218BE09B60F9219BE16
S11324800BB60F921BBE2F933F934F935F936F93A3
S11324907F938F939F93AF93BF93CF93EF93FF93C8
S11324A00E9497018091A108887121F00E948C03F9
S11324B00E949F01C091A0080E940C05811105C0D3
S11324C00E9493030E94A30104C08C2F90E00E94F9
S11324D060050E949B01FF91EF91CF91BF91AF9155
S11324E09F918F917F916F915F914F913F912F9128
S11324F00F900BBE0F9009BE0F9008BE0F900FBE39
S11325000F901F9018951F920F920FB60F921124DF
S113251008B60F9218BE09B60F9219BE0BB60F92E9
S11325201BBE2F933F934F935F936F937F938F9330
S11325309F93AF93BF93EF93FF930E9477048823F5
S113254039F00E948F010E94D0048093A00805C036
S113255080E38093A3080E949301FF91EF91BF91C0
S1132560AF919F918F917F916F915F914F913F9127
S11325702F910F900BBE0F9009BE0F9008BE0F90C5
S11325800FBE0F901F9018958FEF8093700080936B
S11325907100809372008093730080937400809321
S11325A07500809376000895CF93DF931F92CDB783
S11325B0DEB79FB79983F8949981E82FF0E0E0594A
S11325C0FF4F60958081682360839FBF0F90DF91E8
S11325D0CF910895CF93DF931F92CDB7DEB79FB706
S11325E09983F8949981E82FF0E0E059FF4F8081B6
S11325F0682B60839FBF0F90DF91CF910895CF9395
S1132600DF93FC01709620E030E0C62FD0E0DE01BD
S1132610022E02C0B595A7950A94E2F7A0FD508357
S11326202F5F3F4F31962830310589F740FF0AC0AC
S113263041FF03C0FC01658302C0FC016683FC0109
S1132640618302C0FC016283DF91CF91089543E06E
S113265050E061E080E096E00E94FF1243E050E029
S113266062E080E096E00E94FF1243E050E064E004
S113267080E096E00E94FF1243E050E068E080E0D2
S113268096E00E94FF1243E050E060E180E096E0B3
S11326900E94FF1243E050E060E280E096E00E9476
S11326A0FF1243E050E060E480E096E00E94FF12F5
S11326B043E050E060E880E096E00E94FF1240E0D2
S11326C058E161E080E296E00E94FF1240E058E1A8
S11326D062E080E296E00E94FF1240E058E164E08C
S11326E080E296E00E94FF1240E058E168E080E258
S11326F096E00E94FF120895AA1BBB1B51E107C07C
S1132700AA1FBB1FA617B70710F0A61BB70B881F7D
S1132710991F5A95A9F780959095BC01CD0108950C
S1132720A1E21A2EAA1BBB1BFD010DC0AA1FBB1FD1
S1132730EE1FFF1FA217B307E407F50720F0A21B43
S1132740B30BE40BF50B661F771F881F991F1A94B0
S113275069F760957095809590959B01AC01BD01DA
S1132760CF010895EE0FFF1F881F8BBF0790F691CE
S1132770E02D1BBE1994FB01DC0102C001900D92F7
S10F278041505040D8F70895F894FFCF62
S113278C12042F03BA01BC01C102C401B4013B03FE
S113279CBC01000066201A20000022201E200A2002
S11327AC002009024300020100C0320904000001A8
S11327BC020201000524001001042402020524066F
S11327CC00010524010301070582034000100904DC
S11327DC0100020A00000007058102400000070501
S11327EC0202400000001201000202000040EB0350
S11327FC0424000101020001000300000000000099
S113280C00000000000000000000000000000000B8
S113281C0000000000000000434443205669727419
S113282C75616C20436F6D0041544D454C204153F0
S109283C46000403090438
S9030000FC
